:020000007E2957
:08000800FF0003088301FE0064
:100010000408FD008029A501AF00B001A01125084A
:100020000319A0150430A400300E1B2030081B203B
:100030002F0E1B202F080F39F63E0318073E0A3EED
:100040004128A501AF00B001A01125080319A01592
:100050000530A4002730AE0010303A200330AE0047
:10006000E8303A20AE0164303A20AE010A303A203E
:100070002F084128AD003008AC002F08AB00472105
:100080002B08AB00A4030319A011250803194B2862
:100090002402031852282B08031DA011A01952286E
:1000A000303E0B290800B200851105118316851119
:1000B00005110F30860583123208A0187D283E30C6
:1000C000AC00803033213330B10091201330AC00CC
:1000D00088303321912064303221912064303221E4
:1000E0002230B100912028307C200C307C2006305A
:1000F0007C20A01432087D282014B100201C8B28FD
:100100000511033C031C902890200530AC00DC3026
:100110003321031408002014FE3C03199E28051502
:10012000201C201085150F3086053108F039860413
:100130008511B10E201891283230322132087929E8
:100140002016201E2012A01AA928A016DF200318AE
:10015000D42820110830AE00F020AD0DAE0BAC2835
:100160002019B928201AB5280621FF20FB20201AC3
:10017000D420032103102D08DB282016201E201276
:10018000201BC728FE39A60020170310DB28A01B60
:10019000CF28B100A017DF200318D4283108E320AE
:1001A0000318D428201EDB280621FF202013A013CB
:1001B000A012201103213314031C33107929F820D5
:1001C0002608A01A0138AD000830AE00AD0D03219D
:1001D0000318EB280621FF20FB20AE0BE6280321A5
:1001E000FF20F2286400031005180314FB20080008
:1001F0000321FF2006218510831685100929851407
:1002000083168510092983160514092905108316FC
:10021000051083120800A11B5328A11C11292118C5
:10022000BF2883169B0083161C141A089B0A792981
:1002300083169A001C1555309D00AA309D009C1411
:100240009C1820291C119B0A7929AE01AD00FF30B2
:10025000AD07031CAE07031C79290330AC00DF3067
:1002600033212729AC01E83EAB00AC09FC30031C6C
:100270003C29AB0703183929AB070000AC0F39291B
:100280002B184229AB1C4629000046290800B00162
:10029000AF011030B1002C0DAF0DB00D2D08AF0225
:1002A0002E08031C2E0FB00203185D292D08AF077E
:1002B0002E0803182E0FB0070310AB0DAC0DB10BB9
:1002C0004B292B0879291030B500AC01AB01B20CD9
:1002D000B10C031C71292D08AB072E0803182E0F33
:1002E000AC07AC0CAB0CB00CAF0CB50B67292F08EE
:1002F000792983138312031300000800A0018F29BA
:1003000006188629861D3F148619BF1410308B00ED
:100310007D0884007E088300FF0E7F0E09008B138A
:1003200007309F007030831685000F3086008101F2
:1003300010308B008312D201CC01CB01E1010130DE
:10034000C10003011121C2001321C3000230112199
:10035000C4001321C50004301121D2000530112141
:10036000CA0050301121C8001321C9005230112198
:10037000D00053301121D10054301121C00055302C
:100380001121CD0058301121D9001321DA005A3043
:100390001121DB001321DC005C301121DD00132171
:1003A000DE005E301121DF001321E0008B17BD2637
:1003B000ED26643025218A27FE305320013053205A
:1003C00032302521FE3053208030532053305320CB
:1003D000613053206C3053207530532074305320DB
:1003E0006930532020305320643053206130532033
:1003F000203053204930532057305320323053207F
:100400004B3053204730532048305320FE30532088
:10041000C0305320413053205430532056305320A5
:1004200020305320532053305320693053206E30F6
:1004300053205330532068305320203053205630FF
:1004400053205F305320323053203130532020303E
:1004500053200730AE0008302621051A302A012B20
:100460000619332AA32BA52A4114BD26E624FE3003
:100470005320C03053208926212714303B05A80182
:10048000A70028082704031D462A4D2A381C492A9C
:10049000C624B81C4C2ACE24652A4C08013C031CF7
:1004A000572A02308A004C088207572AA72A401D83
:1004B0005A2ABB2A381C5D2A702CB81C602A882C4A
:1004C00008303902031D652AB32A10303902031D92
:1004D0006A2ACA0A04303902031D6F2AD72C043055
:1004E0003C02031D742ACE2410303C02031D792ADD
:1004F000C62414303C02031D7E2AC62A143038025A
:10050000031D832AC1140C303802031D882AFC2ADB
:1005100018303802031D8D2AF72A1C303B02031DB8
:10052000922A7F29CA305102031D972A352A401189
:100530004A18A42A08303C02031DA42A5B303E025C
:10054000031CA42A4015CC01352ACC01342A381CBE
:10055000AA2AA024B81CAD2AB32408303902031DEE
:10056000B22AA52A652ACA305102031DB82A352AA3
:100570000130CC00342A381CBE2AA024B81CC12A61
:10058000B3244508C3004408C200652AC11464307E
:100590003E020318CC2A352AFE305320C0305320A7
:1005A0002030532053305320743053206F30532069
:1005B0007230532065305320203053204530532073
:1005C00073305320653053206730532075305320EB
:1005D00069305320743053206F3053202030532023
:1005E0003A2621273B080319F62AF12A352A8030BA
:1005F000D2060630C104352A0130D2060630C104C5
:10060000352A4114FE305320C0305320523053203D
:100610008030A10050080B2020305320543053204C
:100620008030A10051080B20203053204F30532040
:100630004C305320C0181F2B2B305320212B2D3032
:1006400053204908D4004808D300F225FE30532037
:100650008030532046305320753053206E30532065
:1006600020305320401C3F2B44305320493053202E
:10067000413053204C30532020305320492B5030F0
:100680005320553053204C305320533053202030CA
:10069000532021270130D7003B1E502B1430D700A8
:1006A000381C562B5708C8070318C90AB81C5C2BFE
:1006B0005708C802031CC90308303902031D612B07
:1006C0007C2B10303902031D662B8B23043039023A
:1006D000031D6B2B942314303802031D712B013042
:1006E000C00604303C02031D792B0230C0060630E0
:1006F000C1040A302521022B50085102031D812B11
:10070000022BC2305002031D8A2BC830510203183D
:100710008A2B022B6E2E0230D007C7305002031CEA
:10072000932BC030D00008000230D107C2305102F4
:10073000031D9C2BC630D100CB305102031CA22BD1
:10074000C030D10008002127FE30532080305320D4
:1007500052305320583053205F30532020305320E4
:100760008030A100A5015A08B0005908AF0024202C
:10077000203053205320A5015C08B0005B08AF0077
:100780002420203053205320FE305320C0305320EB
:1007900054305320583053205F30532020305320A2
:1007A0008030A100A5015E08B0005D08AF002420E4
:1007B000203053205320A5016008B0005F08AF002F
:1007C000242020305320532004306102031CE92BE5
:1007D000E1016108031DEE2B8830D8000130610271
:1007E000031DF42B8F30D80002306102031DFA2B59
:1007F000C830D80003306102031D002CCF30D80070
:10080000FE305320580853202A3053200830D70098
:100810003B1E0C2C5030D700381C0F2C1B24B81C4E
:10082000122C3524381D152CE10AB81D182C4F2C1C
:100830001E302521A32B0310610D593E84000008B2
:10084000A900840A0008AA0057082907A7002A0857
:100850000318013EA8000310610D593E84002708CB
:100860008000840A2808800008000310610D593EAA
:1008700084000008A900840A0008AA005708290279
:10088000A7002A08031CFF3EA8000310610D593E73
:10089000840027088000840A280880000800583057
:1008A00083169B008312590818215A0818215A30C0
:1008B00083169B0083125B0818215C0818215C30AA
:1008C00083169B0083125D0818215E0818215E3094
:1008D00083169B0083125F08182160081821A52A3F
:1008E000C01C752C4A1C752C8D2C4D08C207031892
:1008F000C30A43085C02031C832C031D872C420897
:100900005B020318872C5A08C3005908C200352A15
:10091000C01C8D2C4A1C8D2C752C4D08C202031C4A
:10092000C3035A084302031C9B2C031D9F2C590828
:10093000420203189F2C5C08C3005B08C200352AE2
:100940004D08C4070318C50A45086002031CAE2CF5
:10095000031DB22C44085F020318B22C5E08C500C8
:100960005D08C40008004D08C402031CC5035E08EE
:100970004502031CC12C031DC52C5D08440203184D
:10098000C52C6008C5005F08C40008004114CB0AEC
:100990000A304B02031CCD2CCB01512E4114CB034A
:1009A0000B304B02031CD62C0930CB00512E031008
:1009B000CD0D51304D02031CDF2C0230CD0009302B
:1009C0004D02031CE52C5030CD00352A4308C700EA
:1009D0004208C6004608D3004708D4000330AB00E5
:1009E0000310D40CD30CAB0BF02C4A1C082DC018F0
:1009F000002D4808D30749080318013ED407082DE5
:100A000053084802D3005408031C013E4902D40095
:100A1000FE30532080305320523053208030A100CC
:100A20004B0821204C08031D182D2A3053201A2D65
:100A300020305320F2250F264E1E252D2030532026
:100A40003F30532020305320342DCE1E2E2D203009
:100A500053202130532020305320342D4D3053204B
:100A60006830532020305320D21B392D4130532081
:100A70003B2D423053205218402D4E305320422DF2
:100A800057305320FE305320C03053204508C70054
:100A90004408C6004608D3004708D4000330AB0022
:100AA0000310D40CD30CAB0B502DCA305102031DD4
:100AB0005A2DC22D543053208030A1004B082120E4
:100AC00001304C02031D672D2A3053206E2D401D2E
:100AD0006C2D2A3053206E2D20305320F2250F2606
:100AE0004E1C772D203053203F3053207B2D4D302E
:100AF000532068305320CE1C802D21305320822D6E
:100B00002030532002304D02031D8A2D2E305320F9
:100B10003230532004304D02031D922D2E305320CD
:100B20003530532008304D02031D9A2D20305320BC
:100B30003130532050304D02031DA22D313053204F
:100B4000303053200800FE305320943053202030A2
:100B500053208030A1000230A5003B080C2020303B
:100B600053200230A50038080C20203053200230DA
:100B7000A5003C080C20203053200230A5003E0880
:100B80000C2008005330532065305320743053201C
:100B900020305320BB19DE2D2030532053204F30FE
:100BA00053204C30532020305320532053205330B7
:100BB00053205030532020305320F12D203053202B
:100BC000413053202F3053204230532020305320C7
:100BD00053204E3053202F30532057305320203095
:100BE0005320822D03305402E830031953020318B6
:100BF000FB2D2030532027305402103003195302AC
:100C00000318042E203053208030A100A501540881
:100C1000B0005308AF0024202E30532008004708AE
:100C2000B7004608B6000730B605B7010310B70C89
:100C3000B60C3708B2003608B100AE011930AD006D
:100C40006321D3003008D400D308031D2A2ED40812
:100C50000319322E8030A100A5015408B0005308BA
:100C6000AF00242054085304031D392E3030532084
:100C7000532008006726580883169B0083124208F9
:100C80001821430818214408182145081821520842
:100C900018214A081821553083169B0083124D08ED
:100CA0001821C114672658081121C2001321C3005E
:100CB000023058071121C4001321C5000430580721
:100CC0001121D200053058071121CA000800031075
:100CD0004B0D4B07D8000310D80D08005030831679
:100CE0009B008312480818214908182152308316A6
:100CF0009B00831250081821533083169B008312E7
:100D000051081821543083169B0083124008182183
:100D1000A52A0F30CE055008BF20A020D800331CD4
:100D2000932E4E16962E581B962ECE164330430207
:100D3000031CA92E031DA02E31304202031CA92E34
:100D4000FC304202D3000E30031C013E4302D400AB
:100D5000B12EFC304207D3000E300318013E43078A
:100D6000D4005008BF205408BF205308BF20CE3005
:100D7000BF205208BD20D4200800F030CE05CA3074
:100D80005102031DC42E0800C8305102031DC92E94
:100D9000ED2E5108BF20A020D800331CD12E4E14B8
:100DA000CF01581BD52ECF0AD62ECF0115304F02BA
:100DB000031CDC2ECE14CF034508D4004408D30016
:100DC0005108BF205408BF205308BF20CE30BF2099
:100DD0005208BD208517D4200800D4200514703097
:100DE000831685008312D401D301441A5314C41A04
:100DF000D314441B5315C41BD31545185316C518DB
:100E0000D31645195317C519D31744195414C419C7
:100E1000D4140130D700113057020318192F851050
:100E2000D30DD40D03180514031C05108514D70F1A
:100E30000B2F85130430AB00AB0B1C2F8517D42070
:100E4000080005302521B80140182C2F8619292FBC
:100E5000381406182C2FB81406192F2F3815051A18
:100E6000322FB8158618352F3816411C3A2FBD0180
:100E7000BE01BB01B9013808031D472FBD01BE01EA
:100E8000C11C432FBA01C1013A08B900BA01411D82
:100E90004A2FBE0138083B020319502FBD01BE0185
:100EA0003808BB00B801BC01BD0ABE0A03303D02D0
:100EB000031D5C2F3B08B80004303D02031C622F69
:100EC0003B08BA002E303D02031C682F3B08B800D7
:100ED00033303E02031C6E2F3B08BC002E303D0217
:100EE000031C742F2C30BD00FB303E02031C7A2FF4
:100EF000FA30BE00401C892FFC30B80501303F029B
:100F0000031D832F381402303F02031D882FB814AD
:100F1000BF010800FE30532003015320FE30532050
:100F200020305320FE30532028305320FE305320F1
:100F30000C305320FE30532006305320FE30532017
:0A0F40001430532008006300A32FB3
:02400E00503F21
:10420000C0002600B000260000000100C00026000B
:10421000B400260000000000C0002600B800260000
:1042200000000100C0002600BC00260000000000C5
:10423000C0002600C000260000000000C0002600CC
:10424000C400260000000100C0002600C8002600AF
:1042500000000000C0002600CC0026000000000086
:10426000C0002600D000260000000100C00026008B
:10427000D40026000000000040001F008000250040
:104280000000000040001F0080002500000000002A
:10429000000000000000000000000000000000001E
:1042A000B8002400C600C0000100080000000000A3
:1042B00000001900A000410040001F00E0002E0097
:00000001FF
